:020000000150AD
:02000B0021AE24
:10005000C20075B0FF7590FF75816F758912754B81
:1000600000754C00754D00754E00C201C202C203FE
:10007000C204C206C20575453275466475471975D6
:1000800048C8754AFA758C38C28ED28CD2A9D2AFC4
:1000900075410175442075430D7542208000200094
:1000A0000D30B0057548C8C20430046CD200200180
:1000B00011E54B600D754021854049D203754F0114
:1000C000D20120061CE54CB40117E54BB4011275B2
:1000D00048C8C20475400A854049D203754F01D211
:1000E0000630061FE54CB4000BE54BB40606D205FE
:1000F000C2AF015030B0057548C8C204300404C214
:10010000AF01520031232001043151019E20060429
:10011000315E019E3191019E75421F7543207544E9
:1001200020019E30022AC202054EE54EB40A217516
:100130004E00054DE54DB40617754D00054CE54CD8
:10014000B40A0D754C00054BE54BB40A03754B0022
:1001500022E54C4410F542854D43854E4422300340
:100160002FC203D54F03754F0A740AC3954F23233B
:10017000FF90024893F5420FEF93F5430FEF93F58D
:10018000440FEF93F5502540FFC3940340028F4086
:1001900022854B43854C44300313C203D54F03756E
:1001A0004F087408C3954F90027093F54222C0E047
:1001B000C0D0C082C083300016D54513754532D5F6
:1001C0004905854049D203D54605754664D202D516
:1001D0004745754705D54805854A48B20490022031
:1001E000D54103754103759000D2B5D2B4D2B7D2D0
:1001F000B3E541B40109E54493F590C2B58018B464
:100200000209E54393F590C2B4800CB40309E542BA
:1002100093F590C2B78000D083D082D0D0D0E032A6
:10022000FA9079D993CBEB98FBDB85C46425000069
:10023000FE947DDD97CFEF9CFFDF8444240500040E
:10024000000A0818C040602221202000222220003D
:100250002022220020202300202001002020240032
:10026000202525002525200026202000272020FFEE
:080270000A1A0B1B0C1C0D1DEA
